S01E000062696E2F64656D6F70726F675F73746D3332683734332E7372656323
S3150802000000000220B10702080108020801080208D6
S315080200100108020801080208010802080000000097
S3150802002000000000000000000000000001080208AD
S31508020030010802080000000001080208353F02080C
S315080200400108020801080208010802080108020854
S315080200500108020801080208010802080108020844
S315080200600108020801080208010802080108020834
S315080200700108020801080208010802080108020824
S315080200800108020801080208010802080108020814
S315080200900108020801080208010802080108020804
S315080200A001080208010802080108020801080208F4
S315080200B001080208010802080108020801080208E4
S315080200C001080208010802080108020801080208D4
S315080200D001080208010802080108020801080208C4
S315080200E001080208010802080000000001080208C7
S315080200F001080208010802080108020801080208A4
S315080201000108020801080208010802080108020893
S315080201100108020801080208010802080108020883
S315080201200108020801080208010802080108020873
S315080201300108020801080208010802080108020863
S31508020140000000000000000000000000000000009F
S315080201500108020801080208010802080108020843
S315080201600108020801080208010802080108020833
S315080201700108020801080208010802080000000036
S315080201800108020801080208010802080108020813
S315080201900108020801080208010802080108020803
S315080201A001080208010802080108020801080208F3
S315080201B001080208010802080108020801080208E3
S315080201C001080208010802080108020801080208D3
S315080201D001080208010802080108020801080208C3
S315080201E001080208010802080108020801080208B3
S315080201F001080208010802080108020801080208A3
S315080202000108020801080208010802080108020892
S315080202100108020801080208010802080108020882
S315080202200108020801080208010802080000000085
S315080202300108020801080208000000000108020875
S315080202400108020801080208010802080108020852
S315080202500108020801080208010802080108020842
S315080202600108020801080208010802080108020832
S315080202700108020801080208010802080000000035
S315080202800108020801080208010802080000000025
S311080202900000000001080208EE11AA5541
S315080202A010B5054C237833B9044B13B10448AFF3A0
S315080202B000800123237010BD3C04002000000000CA
S315080202C07844020808B5034B1BB103490348AFF348
S315080202D0008008BD0000000040040020784402089F
S315080202E053B94AB9002908BF00281CBF4FF0FF318D
S315080202F04FF0FF3000F074B9ADF1080C6DE904CE89
S3150802030000F006F8DDF804E0DDE9022304B07047E0
S315080203102DE9F047089E04468846002B40F0858062
S315080203208A42154648D9B2FA82F24AB1C2F1200780
S3150802033001FA02F320FA07F7954047EA03089440C0
S315080203404FEA154E230CB8FBFEF71FFA85FC0EFB87
S31508020350178843EA084307FB0CF1994209D9EB18B7
S3150802036007F1FF3080F0E380994240F2E080023FD5
S315080203702B445B1AA4B2B3FBFEF00EFB103344EA1D
S31508020380034400FB0CFCA44509D92C1900F1FF33E0
S3150802039080F0CB80A44540F2C88002382C4440EA5B
S315080203A00740A4EB0C0400271EB1D4400023C6E97B
S315080203B000433946BDE8F087002A53D0B2FA82F2E2
S315080203C0002A40F0B680491B4FEA154E1FFA85F8F7
S315080203D00127B1FBFEFC230C0EFB1C1143EA014369
S315080203E008FB0CF1994207D9EB180CF1FF3002D23F
S315080203F0994200F2EC808446591AA3B2B1FBFEF088
S315080204000EFB101443EA044408FB00F8A04507D97A
S315080204102C1900F1FF3302D2A04500F2DC801846FF
S31508020420A4EB080440EA0C40BEE78B4208D9002E2A
S3150802043078D00027C6E9000138463946BDE8F08774
S31508020440B3FA83F77FB98B4202D3824200F2BD80A8
S31508020450841A61EB030301209846002EA9D0C6E947
S315080204600048A6E7FFDEC7F12005BB4022FA05FCD5
S315080204704CEA030C01FA07F420FA05F821FA05F307
S315080204804FEA1C4E48EA0404B3FBFEF9210C0EFBA4
S3150802049019331FFA8CF841EA034309FB08FA9A450D
S315080204A002FA07F200FA07F10BD91CEB030309F16A
S315080204B0FF3080F088809A4540F28580A9F10209CA
S315080204C06344A3EB0A03A4B2B3FBFEF00EFB10339C
S315080204D044EA034400FB08F8A04508D91CEB0404C7
S315080204E000F1FF336BD2A04569D90238644440EA69
S315080204F00940A4EB0804A0FB02894C45C6464B46B4
S3150802050054D351D0002E69D0B1EB0E0264EB03042A
S3150802051004FA05F522FA07F3FC401D43C6E900541E
S31508020520002746E73746304643E7184637E7074681
S315080205301FE7C2F1200320FA03F7954001FA02F0F9
S3150802054021FA03F34FEA154E3843010CB3FBFEF7C3
S315080205501FFA85F80EFB173341EA034107FB08F336
S315080205608B4204FA02F407D9691807F1FF3C28D22C
S315080205708B4226D9023F2944CB1A81B2B3FBFEF03D
S315080205800EFB103341EA034100FB08F38B4207D9FD
S31508020590691800F1FF3C10D28B420ED90238294461
S315080205A0C91A40EA074714E74145ABD2B8EB020E2F
S315080205B069EB0C0201381346A4E76046F0E71846D1
S315080205C095E76746D8E781467BE7384645E7ACF1C3
S315080205D0020C2B4410E702382C4421E73746E8E69A
S315080205E0704700BF70B50D4E0D4D761BB61006D07E
S315080205F00024013455F8043B9847A642F9D1094E1E
S31508020600094D761B03F038FFB61006D000240134D4
S3150802061055F8043B9847A642F9D170BD2C45020805
S315080206202C450208344502082C450208F0B4860710
S3150802063046D0541E002A3CD0CAB2034602E014F140
S31508020640FF3436D303F8012B9D07F8D1032C29D999
S31508020650CDB245EA05250F2C45EA054533D9A4F15D
S315080206601006360903F1200707EB061703F11002F5
S3150802067042E9045542E902551032BA42F8D1721CCF
S3150802068014F00C0F03EB021204F00F0613D0331FFB
S3150802069023F003030433134442F8045B9342FBD169
S315080206A006F003042CB1C9B21C4403F8011B9C4290
S315080206B0FBD1F0BC704734461346002CF3D1F8E759
S315080206C014460346C2E71A462646E0E7024B13B12A
S315080206D0024800F005B8704700000000ED0602085F
S315080206E0002301461A46184600F01EB838B50A4CC9
S315080206F00A4D641BA4100AD004F18043013B05EBA2
S315080207008305013C55F804399847002CF9D1BDE810
S31508020710384003F0B7BE00BF384502083445020820
S31508020720704700BF704700BF2DE9F0411E4C0546D1
S31508020730206890461F460E46FFF7F2FF1B4B1A68C3
S31508020740D2F8483133B35A6820681F2A27DC4DB9D4
S31508020750911C01325A6043F82160FFF7E3FF00203B
S31508020760BDE8F08103EB82010124C1F8888004FA0E
S3150802077002FED3F88841022D44EA0E0CC3F888C15A
S31508020780C1F80871E4D1D3F88C114EEA0104C3F812
S315080207908C41DDE702F5A673C2F84831D3E7FFF7C5
S315080207A0C1FF4FF0FF30DBE728040020DC440208D3
S315080207B0DFF834D0002103E00C4B5B584350043178
S315080207C00B480C4B42189A42F6D30B4A02E0002316
S315080207D042F8043B094B9A42F9D300F013F8FFF7A3
S315080207E001FF03F051FC7047000002203845020859
S315080207F0000000203C0400203C040020FC050020E8
S31508020800FEE70000184AD2F8883043F47003C2F8AB
S315080208108830164B1A6842F001021A6000221A61E1
S3150802082018681349014019609A61DA611A629A6274
S31508020830DA621A635A639A63DA631A645A6419683B
S3150802084021F4802119601A660A4B1A680A4B13406A
S31508020850B3F1005F02D2094B01221A60024B4FF034
S3150802086000629A60704700BF00ED00E0004402583B
S315080208707FEDF6EA0010005C0000FFFF08810051D8
S31508020880654B1B6903F03803102B00F0C380182B45
S315080208901CD0A3B1614A60488369C3F30323604944
S315080208A0CB5CDA40836903F00F03CB5C03F01F03CA
S315080208B022FA03F35B490B605B4B1A607047564B8F
S315080208C01B68C3F3C103594ADA40E4E75249886A06
S315080208D000F003008A6AC2F30512CB6A03F0010329
S315080208E0496BC1F3CC0103FB01F307EE903AF8EE2C
S315080208F0677A002ACFD0012852D0F0B102286CD0EC
S3150802090007EE102AF8EE476A9FED496A86EE267ABE
S31508020910414B1B6BC3F3080306EE903AF8EE666A80
S315080209209FED446A67EE867A76EEA77AF7EE006A54
S3150802093077EEA67A27EE277A22E037480168C1F3CE
S31508020940C1013A4BCB4007EE103AF8EE476A07EE7A
S31508020950102AB8EE476A86EE867A036BC3F3080353
S3150802096006EE903AF8EE666A9FED326A67EE867A86
S3150802097076EEA77AF7EE006A77EEA67A27EE277A58
S31508020980254B1B6BC3F34623013307EE903AF8EE69
S31508020990677AC7EE276AFCEEE67A17EE902A7AE7B6
S315080209A007EE102AF8EE476A9FED216A86EE267A46
S315080209B0194B1B6BC3F3080306EE903AF8EE666A08
S315080209C09FED1C6A67EE867A76EEA77AF7EE006ADC
S315080209D077EEA67A27EE277AD2E707EE102AF8EEFE
S315080209E0476A9FED156A86EE267A0B4B1B6BC3F395
S315080209F0080306EE903AF8EE666A9FED0E6A67EE0F
S31508020A00867A76EEA77AF7EE006A77EEA67A27EE68
S31508020A10277AB5E7094A3EE70044025800093D002D
S31508020A20E0440208300400202C0400200090D00381
S31508020A300024744A000000390024F44A00127A009D
S31508020A40104B1B780BB90120704710B504464FF4BA
S31508020A507A70B0FBF3F30C4A1068B0FBF3F001F0BE
S31508020A60E5FB68B90F2C01D901200AE000222146CC
S31508020A704FF0FF3001F0A8FB044B1C60002000E099
S31508020A80012010BD340400202C0400203804002064
S31508020A9010B5032001F086FB01F0FEF80F498B69B9
S31508020AA0C3F303230E4AD35C03F01F03D8408B69B2
S31508020AB003F00F03D35C03F01F0320FA03F3094A7A
S31508020AC01360094B18600020FFF7BAFF10B1012422
S31508020AD0204610BD044603F0E1FAF9E7004402583D
S31508020AE0E0440208300400202C040020034B1B7843
S31508020AF0034A11680B441360704700BF3404002090
S31508020B00F8050020014B1868704700BFF805002059
S31508020B10014B1868000C70470010005C08B501F01C
S31508020B20FBFA054B1B6AC3F30213044AD35C03F0B0
S31508020B301F03D84008BD00BF00440258E04402081B
S31508020B4010B478498C6A8A6AC2F30532CB6AC3F34F
S31508020B500013C96BC1F3CC0103FB01F3002A00F0B1
S31508020B60DB8004F0030407EE903AF8EE677A012C6C
S31508020B7066D0FCB1022C00F0B28007EE102AB8EE5D
S31508020B80477A9FED696AC6EE076A664B9B6BC3F3A3
S31508020B90080307EE103AB8EE477A9FED646A67EEE5
S31508020BA0867A77EE277AB7EE007A77EE877A66EE56
S31508020BB0A76A61E05B4B1B6813F0200F23D0594CE0
S31508020BC02168C1F3C1015A4BCB4007EE103AB8EE81
S31508020BD0477A06EE902AB8EE666AC7EE066AA36BED
S31508020BE0C3F3080307EE103AB8EE477A9FED4F6A49
S31508020BF067EE867A77EE277AB7EE007A77EE877A05
S31508020C0066EEA76A38E007EE102AB8EE477A9FED35
S31508020C10496AC6EE076A434B9B6BC3F3080307EEA2
S31508020C20103AB8EE477A9FED416A67EE867A77EE12
S31508020C30277AB7EE007A77EE877A66EEA76A1BE01E
S31508020C4007EE102AB8EE477A9FED376AC6EE076AAC
S31508020C50344B9B6BC3F3080307EE103AB8EE477A98
S31508020C609FED326A67EE867A77EE277AB7EE007AD2
S31508020C7077EE877A66EEA76A2A4A936BC3F3462308
S31508020C8007EE103AB8EE477AB7EE006A37EE067AFA
S31508020C90C6EE877AFCEEE77AC0ED007A936BC3F369
S31508020CA0064307EE103AB8EE477A37EE067AC6EEEC
S31508020CB0877AFCEEE77AC0ED017A936BC3F3066393
S31508020CC007EE903AF8EE677A77EE867A86EEA77A94
S31508020CD0BCEEC77A80ED027A5DF8044B704707EEE0
S31508020CE0102AB8EE477A9FED146AC6EE076A0D4BCC
S31508020CF09B6BC3F3080307EE103AB8EE477A9FEDEB
S31508020D000B6A67EE867A77EE277AB7EE007A77EE7F
S31508020D10877A66EEA76AAFE70023036043608360BB
S31508020D20DAE700BF004402580024744A000000397A
S31508020D300090D0030024744C0024F44A10B4784975
S31508020D408C6A8A6AC2F30552CB6AC3F30023496CDA
S31508020D50C1F3CC0103FB01F3002A00F0DB8004F0A7
S31508020D60030407EE903AF8EE677A012C66D0FCB1D6
S31508020D70022C00F0B28007EE102AB8EE477A9FEDF1
S31508020D80696AC6EE076A664B1B6CC3F3080307EE6D
S31508020D90103AB8EE477A9FED646A67EE867A77EE7E
S31508020DA0277AB7EE007A77EE877A66EEA76A61E067
S31508020DB05B4B1B6813F0200F23D0594C2168C1F3F3
S31508020DC0C1015A4BCB4007EE103AB8EE477A06EE07
S31508020DD0902AB8EE666AC7EE066A236CC3F308035E
S31508020DE007EE103AB8EE477A9FED4F6A67EE867AB3
S31508020DF077EE277AB7EE007A77EE877A66EEA76AF3
S31508020E0038E007EE102AB8EE477A9FED496AC6EE31
S31508020E10076A434B1B6CC3F3080307EE103AB8EE96
S31508020E20477A9FED416A67EE867A77EE277AB7EEBA
S31508020E30007A77EE877A66EEA76A1BE007EE102A33
S31508020E40B8EE477A9FED376AC6EE076A344B1B6CD3
S31508020E50C3F3080307EE103AB8EE477A9FED326AF3
S31508020E6067EE867A77EE277AB7EE007A77EE877A92
S31508020E7066EEA76A2A4A136CC3F3462307EE103AAC
S31508020E80B8EE477AB7EE006A37EE067AC6EE877A82
S31508020E90FCEEE77AC0ED007A136CC3F3064307EE5D
S31508020EA0103AB8EE477A37EE067AC6EE877AFCEE3D
S31508020EB0E77AC0ED017A136CC3F3066307EE903A3C
S31508020EC0F8EE677A77EE867A86EEA77ABCEEC77A66
S31508020ED080ED027A5DF8044B704707EE102AB8EEE9
S31508020EE0477A9FED146AC6EE076A0D4B1B6CC3F36D
S31508020EF0080307EE103AB8EE477A9FED0B6A67EEDB
S31508020F00867A77EE277AB7EE007A77EE877A66EEF2
S31508020F10A76AAFE70023036043608360DAE700BF8E
S31508020F20004402580024744A000000390090D00395
S31508020F300024744C0024F44A30B4446B0268D2F894
S31508020F408410704B194041EA8401C2F88410026881
S31508020F50D2F8841021F47F01856B41EA0541C2F873
S31508020F608410826B22440468D4F88810194041EA36
S31508020F708201C4F888100468D4F8881021F4FE01A6
S31508020F80C56B41EA0541C4F88810C16B02EB410200
S31508020F900468D4F8A010194041EA8201C4F8A010E6
S31508020FA00468D4F8A01021F4FE01056C41EA054153
S31508020FB0C4F8A010046C416C01FB04240268D2F840
S31508020FC0B010194041EA8401C2F8B0100268D2F89A
S31508020FD0B01021F4FE01856C41EA0541C2F8B01051
S31508020FE0826CC16C01FB02440268D2F8AC1019404B
S31508020FF041EA8401C2F8AC10026D416D01FB02425E
S315080210000468D4F8F010194041EA8201C4F8F010D5
S315080210100468D4F8F01021F47C11856D41EA054183
S31508021020C4F8F010816D02EB41020468D4F8C010CE
S315080210300B4043EA8202C4F8C0200268D2F8C030E4
S3150802104023F47C13C16D43EA0143C2F8C030026837
S31508021050D2F8C03023F07C53016E43EA0163C2F82A
S31508021060C030436B284A1A449200C266836B02EB6D
S3150802107083030367C16B03EBC1034367046C416CCB
S3150802108001FB04F103EB81038367846CC16C01FBEA
S3150802109004F103EB8103C367046D416D01FB04F19F
S315080210A003EB8103C0F88030816D03EBC103C0F8FE
S315080210B08430C46D856E05FB04F403EB8403C0F823
S315080210C08830016E01FB05F103EB8103C0F890300D
S315080210D00E498B4207D8D0F8903093420ED9002396
S315080210E042F8043BF7E7D0F89C3043F02003C0F8F7
S315080210F09C30032380F89830012000E0002030BCA1
S31508021100704700BF0300FFFF002B0010FCD300400E
S315080211107047000030B595B004464C22A04901A894
S3150802112003F09CF9002C00F0388123689D4A93420B
S3150802113020D094F898300BB32268936923F01003F1
S315080211409361FFF7DFFC054623689A6912F0080FD8
S315080211501AD0FFF7D7FC401B0A28F5D9D4F89C30D9
S3150802116043F00103C4F89C30032384F89830012025
S3150802117015B030BD03F580736360DAE784F89930F9
S315080211802046FFF7C5FFD7E79A6942F001029A613E
S31508021190FFF7B8FC054623689A6912F0010F0FD1CA
S315080211A0FFF7B0FC401B0A28F5D9D4F89C3043F067
S315080211B00103C4F89C30032384F898300120D7E74A
S315080211C09A6942F002029A61237C012B40D0226876
S315080211D0936943F040039361637C012B3ED02268F6
S315080211E0936923F480439361A37C012B3CD0226844
S315080211F0936943F4805393612268936923F4407395
S31508021200A1680B4393612268936923F0A40393614F
S315080212102268136923F010031361E368012B29D0AE
S31508021220002B2CD0022B00F09B802268936943F096
S31508021230800393612268136943F010031361E3681C
S31508021240032B1CD12268936943F02003936116E0AD
S315080212502268936923F040039361BDE72268936984
S3150802126043F480439361BFE72268936923F480536A
S315080212709361C1E72268936943F004039361A36902
S315080212805A1EE369013B1B0243EA4263226A013A98
S3150802129013436269013A216843EA0243CB61A368B0
S315080212A0B3F5407F62D0236E33B12268D2F8C030DC
S315080212B0616E0B43C2F8C030E36D226ED3420DD085
S315080212C02168D1F8C83023F00703A26E14A800EBF0
S315080212D0820252F84C2C1343C1F8C830236C6BB106
S315080212E02168D1F8BC3023F00703626C14A800EB1E
S315080212F0820252F84C2C1343C1F8BC30A36C73B16A
S315080213002168D1F8BC3023F07003E26C14A800EB14
S31508021310820252F84C2C43EA0213C1F8BC30236D00
S3150802132073B12168D1F8BC3023F4E063626D14A866
S3150802133000EB820252F84C2C43EA0223C1F8BC3075
S315080213402268184B9A4222D00023C4F89430C4F873
S315080213509C30012384F898302046FFF7EDFD07E715
S315080213602268936943F02003936188E7A36A013BE5
S31508021370E26A013A43EA0223226B013A43EA02137A
S31508021380626A013A216843EA0243CB608BE76268E4
S31508021390936823F003039360D6E70120E8E600BFCB
S315080213A09044020800A0004090F89830013BDBB256
S315080213B0012B07D9D0F89C3043F00203C0F89C30C1
S315080213C001207047CB680A68D2B9072B0ED08A6803
S315080213D0DB0643EA82730A6943EA02434A6913430C
S315080213E0C26E496842F82130002070470A69CB6903
S315080213F01B0243EA02438A69134343F06053EFE749
S3150802140010B40A6942EA4372072B0ED08C684B69FC
S3150802141043EA8473006F496800EBC10440F831203F
S31508021420636000205DF8044B70478B69F2E710B4DD
S3150802143090F89840E4B2012C09D0D0F89C3043F0D9
S315080214400403C0F89C3001205DF8044B70479200F3
S3150802145042EA011242EA43020168019B1A43C1F8B1
S3150802146080200020F0E790F89830DBB2012B07D0F5
S31508021470D0F89C3043F00403C0F89C300120704732
S31508021480022380F898300268936923F00103936176
S315080214900023C0F89C30184670470000F0B490F854
S315080214A09840E4B2022C40F0BA8040290CD0412977
S315080214B030D0046D8C4253D8D0F89C3043F02003C8
S315080214C0C0F89C300120B1E00468D4F8A05015F4A5
S315080214D0FE0F0CD0D4F8A45015F07F0F0FD1D0F818
S315080214E09C3043F48073C0F89C3001209EE0D0F80B
S315080214F09C3043F02003C0F89C30012096E0D4F8D3
S31508021500A440C4F3052C446F456C0CFB05F504EBAB
S3150802151085042DE00468D4F8B05015F4FE0F0CD0FB
S31508021520D4F8B45015F07F0F0FD1D0F89C3043F49D
S315080215308073C0F89C30012078E0D0F89C3043F0E4
S315080215402003C0F89C30012070E0D4F8B440C4F3FC
S31508021550052C846FC56C0CFB05F504EB850407E0C6
S31508021560C46F456D01FB05F504EB85044FF0000CCD
S31508021570256805F080455560002D2CD12568C5F3F0
S315080215808A451560256805F000559560256805F0B9
S3150802159000451561A588D561656805F47025D5608D
S315080215A0656805F480155561656805F40015956149
S315080215B0E57905F07F0515626568ED0F556204F158
S315080215C008050024D6891A4FBE5DA64208D92E5DA3
S315080215D01E550134F6E7256825F060451560D1E702
S315080215E040290AD041290DD01F290FD802680123A4
S315080215F003FA01F1C2F8981002E00368C3F8A8C01A
S31508021600002013E00368C3F8B8C0F9E701F01F0128
S315080216100268012303FA01F1C2F89C10F0E7D0F838
S315080216209C3043F00803C0F89C300120F0BC704798
S31508021630F0440208402905D00368D3F8B40000F044
S315080216407F0070470368D3F8A40000F07F00704754
S31508021650134BDB6813F0040F07D1114BDB6803F059
S31508021660070383421AD00120704710B50C4AD36883
S3150802167023F007031843D060FFF744FA0446084BE1
S315080216805B6813F4005F07D1FFF73CFA001BB0F55D
S315080216907A7FF4D9012000E0002010BD00207047AF
S315080216A000480258002800F0DC8238B50446036870
S315080216B013F0010F25D0A94A136903F03803926A79
S315080216C0102B15D0182B0FD06368B3F5803F3ED088
S315080216D0002B52D1A14B1A6822F480321A601A687A
S315080216E022F480221A6037E002F00302022AEBD1C2
S315080216F09A4B1B6813F4003F03D06368002B00F073
S31508021700B282236813F0020F77D0944A1369926A59
S3150802171013F038035AD0182B55D0E368002B00F083
S31508021720B2808E490A6822F0190213430B60FFF74A
S31508021730E9F90546894B1B6813F0040F40F08B80C4
S31508021740FFF7E0F9401B0228F4D9032092E2834A04
S31508021750136843F48033136063682BB3FFF7D2F937
S3150802176005467E4B1B6813F4003FCAD1FFF7CAF938
S31508021770401B6428F5D903207CE2B3F5A02F09D0D3
S31508021780764B1A6822F480321A601A6822F480228A
S315080217901A60E1E7714B1A6842F480221A601A68E5
S315080217A042F480321A60D7E7FFF7ACF905466B4B6D
S315080217B01B6813F4003FA4D0FFF7A4F9401B642862
S315080217C0F5D9032056E212F0030FA6D1634B1B6824
S315080217D013F0040F03D0E368002B00F04682FFF7EC
S315080217E097F941F2030398422CD85C4A536823F4CA
S315080217F07C33216943EA01335360236813F0100FDF
S3150802180070D0564A136903F03803926A082B52D0ED
S31508021810182B4CD0E369002B00F0A2804F4A1368BC
S3150802182043F080031360FFF76DF905464B4B1B68BF
S3150802183013F4807F7AD1FFF765F9401B0228F5D9A0
S31508021840032017E2454A536823F0FE43216943EA17
S3150802185001635360D1E7FFF75BF941F2030398424C
S3150802186008D83E4A536823F47C33216943EA013394
S315080218705360C2E7394A536823F0FE43216943EAB3
S3150802188001635360B9E7354A136823F0010313600D
S31508021890FFF738F90546314B1B6813F0040FACD035
S315080218A0FFF730F9401B0228F5D90320E2E102F0DE
S315080218B00302012AAED1294B1B6813F4807F03D099
S315080218C0E369802B40F0D381FFF722F941F2030343
S315080218D0984222D8214A536823F0F843216A43EAF8
S315080218E081635360236813F0080F61D06369002B84
S315080218F04AD01A4A536F43F001035367FFF702F9B6
S315080219000546164B5B6F13F0020F51D1FFF7FAF833
S31508021910401B0228F5D90320ACE1104AD36823F00C
S315080219207C53216A43EA0163D360DBE7FFF7F0F8E9
S3150802193041F20303984208D8084A536823F0F84349
S31508021940216A43EA81635360CCE7044AD36823F0E9
S315080219507C53216A43EA0163D360C3E70044025811
S31508021960A74A136823F080031360FFF7CBF80546EE
S31508021970A34B1B6813F4807FB4D0FFF7C3F8401B50
S315080219800228F5D9032075E19D4A536F23F0010316
S315080219905367FFF7B7F80546994B5B6F13F0020FCB
S315080219A006D0FFF7AFF8401B0228F5D9032061E1FC
S315080219B0236813F0200F29D0A3699BB1904A1368B4
S315080219C043F480531360FFF79DF805468C4B1B685A
S315080219D013F4005F1AD1FFF795F8401B0228F5D9D0
S315080219E0032047E1864A136823F480531360FFF7FE
S315080219F089F80546824B1B6813F4005F06D0FFF789
S31508021A0081F8401B0228F5D9032033E1236813F035
S31508021A10040F21D1636A002B00F02B81784A1269E0
S31508021A2002F03802182A00F0F380022B75D0744AA5
S31508021A30136823F080731360FFF764F80446704B4B
S31508021A401B6813F0007F00F0D880FFF75BF8001BD5
S31508021A500228F4D903200DE16A4A136843F4807315
S31508021A601360FFF74FF80546664B1B6813F4807F31
S31508021A7006D1FFF747F8401B6428F5D90320F9E099
S31508021A80A368012B0AD00BBB5D4B1A6F22F0010229
S31508021A901A671A6F22F004021A6704E0584A136F8B
S31508021AA043F001031367A36833B3FFF72BF8054620
S31508021AB0534B1B6F13F0020FACD1FFF723F8401BF1
S31508021AC041F288339842F3D90320D3E0052B09D093
S31508021AD04B4B1A6F22F001021A671A6F22F00402A0
S31508021AE01A67E0E7464B1A6F42F004021A671A6F42
S31508021AF042F001021A67D6E7FFF704F80546404B9B
S31508021B001B6F13F0020F85D0FEF7FCFF401B41F254
S31508021B1088339842F3D90320ACE0394A136823F094
S31508021B2080731360FEF7EEFF0546354B1B6813F00C
S31508021B30007F06D0FEF7E6FF401B0228F5D90320F0
S31508021B4098E02F4B996A304A0A40A16AE06A41EA4C
S31508021B5000110A439A62226B013AC2F30802616BC8
S31508021B600139490289B20A43A16B0139090401F410
S31508021B70FE010A43E16B0139090601F0FE410A43F7
S31508021B801A63DA6A22F00102DA62596B1F4A0A40BC
S31508021B90A16C42EAC1025A63DA6A22F00C02216C8B
S31508021BA00A43DA62DA6A22F00202616C0A43DA62EC
S31508021BB0DA6A42F48032DA62DA6A42F40032DA62C5
S31508021BC0DA6A42F48022DA62DA6A42F00102DA62F8
S31508021BD01A6842F080721A60FEF794FF0446084BB0
S31508021BE01B6813F0007F06D1FEF78CFF001B022844
S31508021BF0F5D903203EE000203CE000203AE000BF91
S31508021C0000440258004802580CFCFFFF0700FFFF79
S31508021C10204A916A106B012B2DD001F00303A26AA8
S31508021C2093422AD1C1F30511E36A994227D1C0F337
S31508021C300802236B013B9A4223D1C0F34622636B07
S31508021C40013B9A421FD1C0F30642A36B013B9A425B
S31508021C501BD1C0F30660E36B013B984217D1002003
S31508021C6008E001207047012004E0012002E001207B
S31508021C7000E0002038BD0120FCE70120FAE7012038
S31508021C80F8E70120F6E70120F4E70120F2E7012050
S31508021C90F0E700BF00440258724B1B6903F0380391
S31508021CA0102B00F0DB80182B10D00BB16E48704752
S31508021CB06C4B1B6813F0200F00F0D280694B186832
S31508021CC0C0F3C100694B23FA00F07047654A916A6E
S31508021CD001F00301906AC0F30510D36A03F0010309
S31508021CE0526BC2F3CC0203FB02F307EE903AF8EE0C
S31508021CF0677A002800F0B580012966D0F9B1022971
S31508021D0000F08F8007EE100AF8EE476A9FED586AD0
S31508021D1086EE267A534B1B6BC3F3080306EE903AFC
S31508021D20F8EE666A9FED536A67EE867A76EEA77ACA
S31508021D30F7EE006A77EEA67A27EE277A61E0494B34
S31508021D401B6813F0200F23D046490A68C2F3C10262
S31508021D50464BD34007EE103AF8EE476A07EE100AEA
S31508021D60B8EE476A86EE867A0B6BC3F3080306EE6D
S31508021D70903AF8EE666A9FED3F6A67EE867A76EEE5
S31508021D80A77AF7EE006A77EEA67A27EE277A38E080
S31508021D9007EE100AF8EE476A9FED376A86EE267A4C
S31508021DA0304B1B6BC3F3080306EE903AF8EE666AED
S31508021DB09FED306A67EE867A76EEA77AF7EE006AC4
S31508021DC077EEA67A27EE277A1BE007EE100AF8EED8
S31508021DD0476A9FED276A86EE267A224B1B6BC3F368
S31508021DE0080306EE903AF8EE666A9FED226A67EEF7
S31508021DF0867A76EEA77AF7EE006A77EEA67A27EE65
S31508021E00277A184B1B6BC3F34623013307EE903A26
S31508021E10F8EE677AC7EE276AFCEEE67A17EE900ABC
S31508021E20704707EE100AF8EE476A9FED146A86EEC7
S31508021E30267A0C4B1B6BC3F3080306EE903AF8EEB0
S31508021E40666A9FED0C6A67EE867A76EEA77AF7EEF1
S31508021E50006A77EEA67A27EE277AD2E7084870470D
S31508021E60024870470044025800093D000090D0031A
S31508021E700024744A000000390024744C0024F44AF1
S31508021E8000127A00002800F0338103469C4A126841
S31508021E9002F00F028A420BD29948026822F00F0218
S31508021EA00A430260026802F00F028A4240F0228167
S31508021EB070B51A6812F0040F0CD01869914A926923
S31508021EC002F07002904205D98E4CA26922F0700285
S31508021ED01043A0611A6812F0080F0CD05869894A93
S31508021EE0D26902F07002904205D9864CE26922F064
S31508021EF070021043E0611A6812F0100F0CD098694C
S31508021F00804AD26902F4E062904205D97D4CE269C0
S31508021F1022F4E0621043E0611A6812F0200F0CD036
S31508021F20D869784A126A02F07002904205D9754C4D
S31508021F30226A22F07002104320621A6812F0020F17
S31508021F400CD0D8686F4A926902F00F02904205D9FE
S31508021F506C4CA26922F00F021043A0611C460D4682
S31508021F601B6813F0010F41D0664A936923F4706324
S31508021F70A1680B4393616368022B0AD0032B27D00F
S31508021F80012B2CD05F4A126812F0040F06D10120E9
S31508021F90ADE0126812F4003F00F0AE8059490A69B2
S31508021FA022F0070213430B61FEF7ACFD0646554BBA
S31508021FB01B6903F038036268B3EBC20F16D0FEF74B
S31508021FC0A1FD801B41F288339842F0D903208EE0A6
S31508021FD04C4A126812F0007FE0D1012087E0494A94
S31508021FE0126812F4807FD9D1012080E0236813F0A9
S31508021FF0020F0CD0E268434B9B6903F00F039A4227
S3150802200005D240498B6923F00F031A438A613C4B78
S315080220101B6803F00F03AB420AD9394A136823F047
S315080220200F032B431360136803F00F03AB4265D10A
S31508022030236813F0040F0CD02269324B9B6903F014
S3150802204070039A4205D22F498B6923F070031A430B
S315080220508A61236813F0080F0CD06269294BDB6981
S3150802206003F070039A4205D22649CB6923F070031E
S315080220701A43CA61236813F0100F0CD0A269214BC8
S31508022080DB6903F4E0639A4205D21E49CB6923F45D
S31508022090E0631A43CA61236813F0200F0CD0E26981
S315080220A0184B1B6A03F070039A4205D215490B6A4C
S315080220B023F070031A430A62FFF7EEFD11498B6992
S315080220C0C3F30323104AD35C03F01F03D8408B697A
S315080220D003F00F03D35C03F01F0320FA03F30B4A42
S315080220E013600B4B18600B4B1868FEF7A9FC70BD02
S315080220F001207047012070470120F8E70120F6E722
S315080221000020005200440258E0440208300400202D
S315080221102C0400203804002008B5FFF7BDFD0B4A41
S315080221209369C3F303230A49CB5C03F01F0320FA1E
S3150802213003F3926902F00F02885C00F01F0023FA8B
S3150802214000F0044A1060044A136008BD00440258AD
S31508022150E0440208300400202C04002008B5FFF7EA
S31508022160DBFF054BDB69C3F30213044AD35C03F0B6
S315080221701F03D84008BD00BF00440258E0440208C5
S3150802218008B5FFF7C9FF054BDB69C3F30223044A07
S31508022190D35C03F01F03D84008BD00BF00440258B1
S315080221A0E04402080649CB6823F4E0631B041B0CCF
S315080221B0000200F4E0600343024A1A43CA60704709
S315080221C000ED00E00000FA0530B4154BDB68C3F3F6
S315080221D00223C3F10704042C28BF04241D1D062D5F
S315080221E001D9033B00E000234FF0FF3505FA04F45A
S315080221F021EA0401994005FA03F322EA0303194383
S31508022200002805DB0901C9B2064B195430BC7047D0
S3150802221000F00F000901C9B2034B1954F6E700BFD3
S3150802222000ED00E000E400E014ED00E00138B0F152
S31508022230807F0AD2064B5860064AF02182F823109C
S315080222400020986007221A6070470120704700BF75
S3150802225010E000E000ED00E0042805D0054A136806
S3150802226023F0040313607047024A136843F0040319
S315080222701360704710E000E0704708B5FFF7FCFFEF
S3150802228008BD0000F0B583B000233AE0092400E057
S315080222900024B4403C4302356E4E46F825406E4C47
S315080222A02568D44304EA05064F6817F4803F01D02F
S315080222B042EA0506684D2E606E6804EA06054F680E
S315080222C017F4003F01D042EA0605634E75604FF0E7
S315080222D0B0452D6804EA05064F6817F4801F01D039
S315080222E042EA05064FF0B0452E606D682C404E68EE
S315080222F016F4001F01D042EA05044FF0B0425460BA
S3150802230001330A6832FA03F400F0A28001249C40E1
S315080223102240F5D04D686E1E112D18BF012E01D927
S31508022320122D12D186685F000325BD4026EA0506EE
S31508022330CD68BD4035438560466826EA04064D6881
S31508022340C5F300149C4034434460C6685F00032505
S31508022350BD40EC4326408D68BD403543C5604D6897
S31508022360122D18BF022D13D1DE08083650F826E0C2
S3150802237003F007054FEA850C0F2505FA0CF52EEA38
S31508022380050E0D6905FA0CF545EA0E0540F82650C4
S31508022390056825404C6804F00304BC402C430460DD
S315080223A04C6814F0805FABD02C4CD4F8F45045F04E
S315080223B00205C4F8F450D4F8F44004F00204019477
S315080223C0019C9D08AE1C234C54F8267003F00304A6
S315080223D0A6000F24B44027EA0407214CA0423FF482
S315080223E057AF04F58064A04222D004F58064A04267
S315080223F020D004F58064A0421ED004F58064A04271
S315080224001CD004F58064A0421AD004F58064A04268
S3150802241018D004F58064A04216D004F58064A04260
S3150802242014D004F58064A0423FF430AF0A2430E7A2
S3150802243001242EE702242CE703242AE7042428E7AA
S31508022440052426E7062424E7072422E7082420E7AA
S3150802245003B0F0BD0004005880000058004402583A
S31508022460000002580AB18161704709048161704708
S3150802247070470000000000002DE9F04387B00446CB
S31508022480016883680269134342691343C2691343A5
S31508022490426E13430868874A02401A430A60226852
S315080224A0536823F44053E1680B435360A1692268D9
S315080224B0814B9A4201D0236A194390687F4B0340A5
S315080224C00B4393602268D36A23F00F03616A0B43B6
S315080224D0D36223687A4A93421FD07A4A934259D0E2
S315080224E0794A934270D0794A934200F08780784AB3
S315080224F0934200F09D80774A934200F0B380764A71
S31508022500934200F0F180754A934200F004816A4AC8
S31508022510934200F0178180252DE1714A526D02F02F
S315080225203802282A34D8DFE812F0290033003300AB
S315080225303300330033003300330025013300330000
S31508022540330033003300330033002B0033003300EB
S31508022550330033003300330033002D0033003300D9
S31508022560330033003300330033002F0033003300C7
S315080225703300330033003300330031000125FAE01B
S315080225800825F8E01025F6E02025F4E04025F2E0DB
S315080225908025F0E0524A526D02F00702052A11D848
S315080225A0DFE812F00600370108000A000C000E00E8
S315080225B00025E0E00825DEE01025DCE02025DAE04B
S315080225C04025D8E08025D6E0454A526D02F007023A
S315080225D0052A11D8DFE812F006001F0108000A00D2
S315080225E00C000E000025C6E00825C4E01025C2E04E
S315080225F02025C0E04025BEE08025BCE0384A526D61
S3150802260002F00702052A11D8DFE812F006000701D0
S3150802261008000A000C000E000025ACE00825AAE016
S315080226201025A8E02025A6E04025A4E08025A2E002
S315080226302B4A526D02F00702052A11D8DFE812F07A
S315080226400600EF0008000A000C000E00002592E0C2
S31508022650082590E010258EE020258CE040258AE0AA
S31508022660802588E01E4A526D02F03802282A39D897
S31508022670DFE802F01538383838383838D738383875
S3150802268038383838173838383838383819383838FA
S31508022690383838381B383838383838381D00012564
S315080226A069E0082567E0102565E0202563E04025F6
S315080226B061E000BFF369FFCF000C0058FFF4FF1179
S315080226C0001001400044004000480040004C004011
S315080226D0005000400014014000780040007C004091
S315080226E000440258802546E0A04A526D02F00702CD
S315080226F0052A0ED8DFE802F003970507090B00251D
S3150802270039E0082537E0102535E0202533E0402555
S3150802271031E080252FE0954A526D02F00702052A1C
S315080227200ED8DFE802F003820507090B002522E02E
S31508022730082520E010251EE020251CE040251AE089
S31508022740802518E002F50E32926D02F00702052A7C
S315080227500ED8DFE802F0036C0507090B02250AE02A
S31508022760082508E0102506E0202504E0402502E0B9
S31508022770802500E004257E4A93425AD0E369B3F5E0
S31508022780004F00F03E85402D01F2CB81DFE815F0BF
S3150802279093070A08C909C9094808C909C909C90913
S315080227A08808C909C909C909C909C909C909C909CB
S315080227B0C808C909C909C909C909C909C909C9097B
S315080227C0C909C909C909C909C909C909C909C90969
S315080227D04809C909C909C909C909C909C909C909DA
S315080227E0C909C909C909C909C909C909C909C90949
S315080227F0C909C909C909C909C909C909C909C90939
S31508022800C909C909C909C909C909C909C909C90928
S3150802281084090425AFE70425ADE70425ABE70425BB
S31508022820A9E70425A7E70425A5E70425A3E70425C0
S31508022830A1E7082D00F0BD800BD9202D00F04F81AD
S31508022840402D00F06A81102D00F0EC80012000F086
S3150802285064BF022D2ED0042D29D103A8FEF770F9E4
S315080228600498636A002B00F08C80012B00F08D809F
S31508022870022B00F08C80032B00F08B80042B00F0D7
S315080228808A80052B00F08980062B00F08880072BAA
S3150802289000F08780082B00F08680092B00F08580DF
S315080228A00A2B00F084800B2B68D001236AE00120F2
S315080228B000F033BFFEF732F9636AD3B1012B42D077
S315080228C0022B42D0032B42D0042B42D0052B42D0F6
S315080228D0062B42D0072B42D0082B42D0092B42D0D6
S315080228E00A2B49D00B2B01D0012303E04FF4807346
S315080228F000E00123B0FBF3F0002801F015816668B9
S3150802290006EB4603834201F21181B0EB063F01F260
S315080229100F81082D00F0548240F26C81202D00F0C0
S315080229206F83402D00F0D183102D00F0A282012082
S315080229300023A3F540710F4A914201F2FB802268F7
S31508022940D36000F0EABE0223D4E70423D2E70623C3
S31508022950D0E70823CEE70A23CCE70C23CAE71023DD
S31508022960C8E72023C6E74023C4E700BF004402584D
S31508022970000C0058FFFC0F008023BBE74FF480735E
S3150802298000E00123B0FBF3F0B6E70223FAE70423DB
S31508022990F8E70623F6E70823F4E70A23F2E70C2307
S315080229A0F0E71023EEE72023ECE74023EAE780234B
S315080229B0E8E76846FEF7C2F90198636AD3B1012BC4
S315080229C01CD0022B1CD0032B1CD0042B1CD0052B8D
S315080229D01CD0062B1CD0072B1CD0082B1CD0092B6D
S315080229E01CD00A2B1CD00B2B01D0012303E04FF479
S315080229F0807300E00123B0FBF3F07DE70223FAE7D8
S31508022A000423F8E70623F6E70823F4E70A23F2E79E
S31508022A100C23F0E71023EEE72023ECE74023EAE74E
S31508022A208023E8E7A94B1B6813F0200F3AD0A74B7F
S31508022A301B68C3F3C103A648D840636AD3B1012B06
S31508022A401CD0022B1CD0032B1CD0042B1CD0052B0C
S31508022A501CD0062B1CD0072B1CD0082B1CD0092BEC
S31508022A601CD00A2B1CD00B2B01D0012303E04FF4F8
S31508022A70807300E00123B0FBF3F03DE70223FAE797
S31508022A800423F8E70623F6E70823F4E70A23F2E71E
S31508022A900C23F0E71023EEE72023ECE74023EAE7CE
S31508022AA08023E8E7636A002B55D0012B55D0022B09
S31508022AB055D0032B55D0042B55D0052B55D0062BB4
S31508022AC055D0072B55D0082B55D0092B55D00A2B94
S31508022AD055D00B2B01D07E480EE77E480CE7636A79
S31508022AE0002B4ED0012B4ED0022B4ED0032B4ED0AC
S31508022AF0042B4ED0052B4ED0062B4ED0072B4ED08C
S31508022B00082B4ED0092B4ED00A2B4FD00B2B01D0B7
S31508022B107148F1E643F60950EEE6636A002B48D09F
S31508022B20012B49D0022B4AD0032B4BD0042B4CD075
S31508022B30052B4DD0062B4ED0072B4FD0082B50D045
S31508022B40092B51D00A2B52D00B2B02D04FF400403E
S31508022B50D2E68020D0E65E48CEE66048CCE66048FB
S31508022B60CAE66048C8E66048C6E66048C4E6604801
S31508022B70C2E65948C0E65F48BEE65F48BCE65F481B
S31508022B80BAE65548B8E65B48B6E65B48B4E65C483A
S31508022B90B2E65A48B0E65B48AEE65B48ACE64D4854
S31508022BA0AAE65A48A8E64FF22440A5E647F61220B6
S31508022BB0A2E64FF400409FE64FF480409CE64FF4AD
S31508022BC0005099E641F2555096E64FF4805093E646
S31508022BD040F6CC4090E640F6AA208DE64FF4006017
S31508022BE08AE64FF4806087E64FF4007084E64FF475
S31508022BF0807081E6022D2FD0042D2AD103A8FDF775
S31508022C009FFF0498636A002B00F0A480012B00F052
S31508022C10B980022B00F0B980032B00F0B980042B8F
S31508022C2000F0B980052B00F0B980062B00F0B980B8
S31508022C30072B00F0B980082B00F0B980092B00F0A9
S31508022C40B9800A2B00F0B9800B2B7FD00122002312
S31508022C5082E0012000236CE6FDF760FF636AE3B1B8
S31508022C60012B55D0022B56D0032B57D0042B58D004
S31508022C70052B59D0062B5AD0072B5BD0082B5CD0D4
S31508022C80092B5DD00A2B5ED00B2B02D00122002322
S31508022C9005E04FF48072002301E00122002300219F
S31508022CA0FDF71EFB0F0247EA106706026268500824
S31508022CB000252B4616EB000847F10009404649460F
S31508022CC0FDF70EFB0346284633E600BF00440258CA
S31508022CD00090D00390D0030000093D000048E801A7
S31508022CE00024F400AAC2A20000127A0000A8610019
S31508022CF05561510080841E0040420F0020A1070042
S31508022D002A2C0A00801A06001516050048E8010052
S31508022D1002220023C3E704220023C0E70622002377
S31508022D20BDE708220023BAE70A220023B7E70C22E6
S31508022D300023B4E710220023B1E720220023AEE7DE
S31508022D4040220023ABE780220023A8E74FF48072D3
S31508022D50002301E0012200230021FDF7C1FA0F0238
S31508022D6047EA106706026268500800252B4616EBEA
S31508022D70000847F1000940464946FDF7B1FA0346FD
S31508022D802846D6E502220023E6E704220023E3E7E3
S31508022D9006220023E0E708220023DDE70A220023B1
S31508022DA0DAE70C220023D7E710220023D4E72022F1
S31508022DB00023D1E740220023CEE780220023CBE777
S31508022DC06846FDF7BBFF0198636AE3B1012B32D06F
S31508022DD0022B33D0032B34D0042B35D0052B36D017
S31508022DE0062B37D0072B38D0082B39D0092B3AD0E7
S31508022DF00A2B3BD00B2B02D00122002305E04FF40D
S31508022E008072002301E0012200230021FDF768FAFF
S31508022E100F0247EA106706026268500800252B4629
S31508022E2016EB000847F1000940464946FDF758FAED
S31508022E30034628467DE502220023E6E7042200230C
S31508022E40E3E706220023E0E708220023DDE70A2259
S31508022E500023DAE70C220023D7E710220023D4E75F
S31508022E6020220023D1E740220023CEE78022002336
S31508022E70CBE7C54B1B6813F0200F5CD0C24B1B680F
S31508022E80C3F3C103C148D840636AE3B1012B34D006
S31508022E90022B35D0032B36D0042B37D0052B38D04E
S31508022EA0062B39D0072B3AD0082B3BD0092B3CD01E
S31508022EB00A2B3DD00B2B02D00122002305E04FF44A
S31508022EC08072002301E0012200230021FDF708FA9F
S31508022ED04FEA012949EA10694FEA002870080025D5
S31508022EE032462B4618EB000649F1000730463946AA
S31508022EF0FDF7F6F9034628461BE502220023E4E716
S31508022F0004220023E1E706220023DEE70822002343
S31508022F10DBE70A220023D8E70C220023D5E7102292
S31508022F200023D2E720220023CFE740220023CCE762
S31508022F3080220023C9E7636AFBB1012B2ED0022B3C
S31508022F4031D0032B34D0042B37D0052B3AD0062B9D
S31508022F503DD0072B40D0082B43D0092B46D00A2B4D
S31508022F6049D00B2B04D0DFF828824FF0030908E07A
S31508022F70DFF818824FF0000903E0DFF814824FF0F9
S31508022F8003097708002532462B4618EB070049F154
S31508022F900001FDF7A5F903462846CAE4DFF8F481DD
S31508022FA04FF00109EDE7DFF8F0814FF00009E8E795
S31508022FB00FF2B419D9E90089E3E7DFF8E0814FF0A7
S31508022FC00009DEE7DFF8D8814FF00009D9E70FF2EA
S31508022FD0A019D9E90089D4E7DFF8C8814FF00009BA
S31508022FE0CFE7DFF8C4814FF00009CAE7DFF8BC81F2
S31508022FF04FF00009C5E7DFF8B8814FF00009C0E7CE
S31508023000636AFBB1012B2ED0022B31D0032B34D0AD
S31508023010042B37D0052B3AD0062B3DD0072B40D0B0
S31508023020082B43D0092B46D00A2B49D00B2B04D0A8
S31508023030DFF870814FF0000908E0DFF878814FF079
S31508023040000903E0DFF85C814FF0000977080025E4
S3150802305032462B4618EB070049F10001FDF740F905
S315080230600346284665E4DFF840814FF00009EDE79C
S31508023070DFF838814FF00009E8E70FF2FC09D9E9D1
S315080230800089E3E7DFF828814FF00009DEE7DFF879
S3150802309028814FF00009D9E70FF2E409D9E9008936
S315080230A0D4E7DFF8E8804FF00009CFE7DFF80C81B4
S315080230B04FF00009CAE7DFF808814FF00009C5E7B3
S315080230C0DFF800814FF00009C0E7636A03B3012BFA
S315080230D030D0022B33D0032B36D0042B39D0052B14
S315080230E03CD0062B74D0072B77D0082B7AD0092B25
S315080230F07DD00A2B00F080800B2B04D04FF40008F9
S315080231004FF0000908E04FF400484FF0000903E0C9
S315080231104FF400084FF000097708002532462B467F
S3150802312018EB070049F10001FDF7DAF803462846CD
S31508023130FFF7FFBB4FF480084FF00009ECE74FF4A6
S3150802314000184FF00009E7E7DFF87C804FF0000926
S31508023150E2E74FF480184FF00009DDE7DFF86C80EC
S315080231604FF00009D8E700BF00AAC2A2000000007B
S315080231700055615100000000002A2C0A00000000D8
S315080231800015160500000000004402580090D003FE
S31508023190000090D0000048E8000024F40000127AEB
S315080231A00000A8610000093D0080841E0040420F0D
S315080231B00020A10700093D0000801A060048E80120
S315080231C00024F40000127A000055150000CC0C0009
S315080231D0DFF8B0854FF000099EE74FF400284FF05C
S315080231E0000999E74FF480284FF0000994E74FF455
S315080231F000384FF000098FE74FF480384FF0000986
S315080232008AE7402D00F25482DFE815F041008F006C
S3150802321052025202CE005202520252020F015202C8
S3150802322052025202520252025202520250015202F1
S3150802323052025202520252025202520252025202DE
S31508023240520252025202520252025202D101520250
S3150802325052025202520252025202520252025202BE
S3150802326052025202520252025202520252025202AE
S31508023270520252025202520252025202520252029E
S315080232805202520252025202520252020C02FEF733
S3150802329065FF636AD3B1012B33D0022B33D0032BDC
S315080232A033D0042B33D0052B33D0062B33D0072B40
S315080232B033D0082B33D0092B33D00A2B33D00B2B20
S315080232C001D0012303E04FF4807300E00123B0FB31
S315080232D0F3F06268530803EB4003B3FBF2F39BB2C5
S315080232E00020A3F110014FF6EF72914200F22484F6
S315080232F09AB222F00F02C3F3420313432268D36041
S315080233000BE20223E3E70423E1E70623DFE70823C8
S31508023310DDE70A23DBE70C23D9E71023D7E72023C7
S31508023320D5E74023D3E78023D1E7FEF729FF636A6F
S31508023330D3B1012B24D0022B24D0032B24D0042B67
S3150802334024D0052B24D0062B24D0072B24D0082BD7
S3150802335024D0092B24D00A2B24D00B2B01D00123ED
S3150802336003E04FF4807300E00123B0FBF3F06268D8
S31508023370530803EB4003B3FBF2F39BB20020B0E71A
S315080233800223F2E70423F0E70623EEE70823ECE735
S315080233900A23EAE70C23E8E71023E6E72023E4E713
S315080233A04023E2E78023E0E703A8FDF7C9FB049B75
S315080233B0626AD2B1012A24D0022A24D0032A24D04E
S315080233C0042A24D0052A24D0062A24D0072A24D05F
S315080233D0082A24D0092A24D00A2A24D00B2A01D062
S315080233E0012203E04FF4807200E00122B3FBF2F2FD
S315080233F061684B0803EB4203B3FBF1F39BB200206F
S315080234006FE70222F2E70422F0E70622EEE7082235
S31508023410ECE70A22EAE70C22E8E71022E6E720228E
S31508023420E4E74022E2E78022E0E76846FDF786FC09
S31508023430019B626AD2B1012A24D0022A24D0032A25
S3150802344024D0042A24D0052A24D0062A24D0072ADE
S3150802345024D0082A24D0092A24D00A2A24D00B2ABE
S3150802346001D0012203E04FF4807200E00122B3FB8F
S31508023470F2F261684B0803EB4203B3FBF1F39BB22A
S3150802348000202EE70222F2E70422F0E70622EEE700
S315080234900822ECE70A22EAE70C22E8E71022E6E726
S315080234A02022E4E74022E2E78022E0E7A34B1B68FA
S315080234B013F0200F42D0A14B1A68C2F3C102A04BE7
S315080234C0D340626AD2B1012A24D0022A24D0032A1E
S315080234D024D0042A24D0052A24D0062A24D0072A4E
S315080234E024D0082A24D0092A24D00A2A24D00B2A2E
S315080234F001D0012203E04FF4807200E00122B3FBFF
S31508023500F2F261684B0803EB4203B3FBF1F39BB299
S315080235100020E6E60222F2E70422F0E70622EEE7B8
S315080235200822ECE70A22EAE70C22E8E71022E6E795
S315080235302022E4E74022E2E78022E0E7636ACBB191
S31508023540012B20D0022B20D0032B20D0042B20D0F5
S31508023550052B20D0062B20D0072B20D0082B20D0D5
S31508023560092B20D00A2B20D00B2B01D0754B02E059
S31508023570754B00E0734B626803EB5203B3FBF2F33D
S315080235809BB20020ADE66E4BF5E7704BF3E7704B46
S31508023590F1E7704BEFE7704BEDE7704BEBE7704BDB
S315080235A0E9E7704BE7E7704BE5E7704BE3E7636AD9
S315080235B0D3B1012B21D0022B21D0032B21D0042BEE
S315080235C021D0052B21D0062B21D0072B21D0082B61
S315080235D021D0092B21D00A2B21D00B2B01D0604BED
S315080235E003E047F6122300E05D4B626803EB5203E1
S315080235F0B3FBF2F39BB2002073E65A4BF5E75A4B3C
S31508023600F3E75B4BF1E7594BEFE75A4BEDE75A4BBA
S31508023610EBE74D4BE9E7594BE7E7594BE5E74FF23D
S315080236202443E2E7636ADBB1012B23D0022B24D0C1
S31508023630032B25D0042B26D0052B27D0062B28D0E2
S31508023640072B29D0082B2AD0092B2BD00A2B2CD0B2
S315080236500B2B02D04FF4803304E04FF4807301E061
S315080236604FF48033626803EB5203B3FBF2F39BB267
S31508023670002036E64FF40043F4E74FF48043F1E7BF
S3150802368042F6AA23EEE74FF40053EBE741F6981306
S31508023690E8E741F25453E5E74FF48053E2E74FF483
S315080236A00063DFE74FF48063DCE74FF40073D9E782
S315080236B00120002315E6FEF751FD636AD3B1012BFB
S315080236C036D0022B36D0032B36D0042B5CD0052BF2
S315080236D05CD0062B5CD0072B5CD0082B5CD0092B60
S315080236E05CD00A2B5CD00B2B01D0012303E04FF4EC
S315080236F0807300E00123B0FBF3F3626803EB520325
S31508023700B3FBF2F39BB20020A3F110014FF6EF725E
S31508023710914200F213822268D3600123A4F86A3028
S31508023720A4F868300023E366236707B0BDE8F08390
S315080237300223E0E70423DEE70623DCE70044025817
S315080237400090D0030020A10720A107000048E80145
S31508023750548545010024F4000050C300AAC2A20001
S3150802376000127A0000093D0080841E0040420F00C4
S315080237705458140000350C002A2C0A0090D0030075
S3150802378048E8010000AA0A000823B4E70A23B2E7B8
S315080237900C23B0E71023AEE72023ACE74023AAE7C1
S315080237A08023A8E7FEF7ECFC636AD3B1012B23D08A
S315080237B0022B23D0032B23D0042B23D0052B23D073
S315080237C0062B23D0072B23D0082B23D0092B23D053
S315080237D00A2B23D00B2B01D0012303E04FF480736D
S315080237E000E00123B0FBF3F3626803EB5203B3FB79
S315080237F0F2F39BB2002087E70223F3E70423F1E7FB
S315080238000623EFE70823EDE70A23EBE70C23E9E7AC
S315080238101023E7E72023E5E74023E3E78023E1E7F0
S3150802382003A8FDF78DF9049B626AD2B1012A23D057
S31508023830022A23D0032A23D0042A23D0052A23D0F6
S31508023840062A23D0072A23D0082A23D0092A23D0D6
S315080238500A2A23D00B2A01D0012203E04FF48072F0
S3150802386000E00122B3FBF2F3626803EB5203B3FBF7
S31508023870F2F39BB2002047E70222F3E70422F1E7BC
S315080238800622EFE70822EDE70A22EBE70C22E9E730
S315080238901022E7E72022E5E74022E3E78022E1E774
S315080238A06846FDF74BFA019B626AD2B1012A23D018
S315080238B0022A23D0032A23D0042A23D0052A23D076
S315080238C0062A23D0072A23D0082A23D0092A23D056
S315080238D00A2A23D00B2A01D0012203E04FF4807270
S315080238E000E00122B3FBF2F3626803EB5203B3FB77
S315080238F0F2F39BB2002007E70222F3E70422F1E77C
S315080239000622EFE70822EDE70A22EBE70C22E9E7AF
S315080239101022E7E72022E5E74022E3E78022E1E7F3
S31508023920874B1B6813F0200F41D0854B1A68C2F3E8
S31508023930C102844BD340626AD2B1012A23D0022A39
S3150802394023D0032A23D0042A23D0052A23D0062AE1
S3150802395023D0072A23D0082A23D0092A23D00A2AC1
S3150802396023D00B2A01D0012203E04FF4807200E033
S315080239700122B3FBF2F3626803EB5203B3FBF2F3E1
S315080239809BB20020C0E60222F3E70422F1E70622F0
S31508023990EFE70822EDE70A22EBE70C22E9E7102215
S315080239A0E7E72022E5E74022E3E78022E1E7636AC8
S315080239B0CBB1012B20D0022B20D0032B20D0042BF5
S315080239C020D0052B20D0062B20D0072B20D0082B61
S315080239D020D0092B20D00A2B20D00B2B01D0594BF3
S315080239E002E0594B00E0574B626803EB5203B3FB04
S315080239F0F2F39BB2002087E6544BF5E7544BF3E704
S31508023A00544BF1E7544BEFE7544BEDE7544BEBE7D6
S31508023A10544BE9E7544BE7E7544BE5E7544BE3E7E6
S31508023A20636AD3B1012B21D0022B21D0032B21D0DB
S31508023A30042B21D0052B21D0062B21D0072B21D0F0
S31508023A40082B21D0092B21D00A2B22D00B2B01D0EF
S31508023A50444B03E043F6095300E0424B626803EB2A
S31508023A605203B3FBF2F39BB200204DE63E4BF5E759
S31508023A703E4BF3E73F4BF1E73D4BEFE73E4BEDE7B6
S31508023A803E4BEBE7304BE9E73D4BE7E74FF2244382
S31508023A90E4E747F61223E1E7636AD3B1012B22D0A2
S31508023AA0022B23D0032B24D0042B25D0052B26D07A
S31508023AB0062B27D0072B28D0082B29D0092B2AD04A
S31508023AC00A2B2BD00B2B02D04FF4004303E08023A2
S31508023AD001E04FF40043626803EB5203B3FBF2F3CF
S31508023AE09BB2002010E64FF48043F4E74FF40053EC
S31508023AF0F1E741F25553EEE74FF48053EBE740F610
S31508023B00CC43E8E740F6AA23E5E74FF40063E2E789
S31508023B104FF48063DFE74FF40073DCE74FF48073FA
S31508023B20D9E701200023EFE50020F6E50120F4E5B8
S31508023B300120F2E50120F0E50120EEE50120ECE5A1
S31508023B40004402580090D00390D003000048E801D0
S31508023B500024F400AAC2A20000127A0000A861009A
S31508023B605561510000093D0080841E0040420F0045
S31508023B7020A107002A2C0A00801A0600151605003D
S31508023B8048E80100836A13F0010F06D002685368F9
S31508023B9023F40033C16A0B435360836A13F0020F9E
S31508023BA006D00268536823F48033016B0B435360D3
S31508023BB0836A13F0040F06D00268536823F480233D
S31508023BC0416B0B435360836A13F0080F06D00268F1
S31508023BD0536823F40043816B0B435360836A13F0E3
S31508023BE0100F06D00268936823F48053C16B0B4307
S31508023BF09360836A13F0200F06D00268936823F451
S31508023C000053016C0B439360836A13F0400F0AD08A
S31508023C100268536823F48013416C0B435360436C68
S31508023C20B3F5801F0BD0836A13F0800F06D00268A3
S31508023C30536823F40023C16C0B4353607047026830
S31508023C40536823F4C003816C0B435360EBE72DE9F9
S31508023C50F04104460F4616469846069D2368DB69D8
S31508023C6037EA03030CBF01230023B3423FD1B5F160
S31508023C70FF3FF3D0FCF746FFA0EB0800A84222D884
S31508023C800DB323681A6812F0040FE7D0DA6912F442
S31508023C90006FE3D04FF400621A622268136823F4B5
S31508023CA0D07313602268936823F00103936020237C
S31508023CB0C4F88030C4F88430C4F88830002384F805
S31508023CC07C30032014E02268136823F4D07313604F
S31508023CD02268936823F0010393602023C4F8803096
S31508023CE0C4F88430002384F87C30032000E00020E6
S31508023CF0BDE8F0812DE9F04383B01E46D0F8843042
S31508023D00202B40F0828004460D469046B2FA82F392
S31508023D105B09002908BF0123002B7AD190F87C3071
S31508023D20012B78D0012380F87C300023C0F8883034
S31508023D302223C0F88430FCF7E5FE0746A4F85C8027
S31508023D40A4F85E80A368B3F5805F06D0A3B922699A
S31508023D5072B9FF22A4F8602014E0226922B940F25F
S31508023D60FF12A4F860200DE0FF22A4F8602009E003
S31508023D707F22A4F8602005E0B3F1805F0AD0002212
S31508023D80A4F86020B4F86080B3F5805F0CD04FF0D9
S31508023D9000091DE022691AB97F22A4F86020F1E71A
S31508023DA03F22A4F86020EDE7236913B14FF000091A
S31508023DB00EE0A94600250BE023685B6A08EA0303BE
S31508023DC029F8023BB4F85E30013B9BB2A4F85E3098
S31508023DD0B4F85E309BB28BB100963B460022202196
S31508023DE02046FFF734FFC0B9002DE5D023685A6A8A
S31508023DF05FFA88F3134005F8013BE3E72023C4F88A
S31508023E008430002084F87C0000E0022003B0BDE87C
S31508023E10F0830120FAE70220F8E70320F6E730B537
S31508023E2083B004460023C0F88830FCF76BFE0546CB
S31508023E3023681B6813F0080F0ED123681B6813F05A
S31508023E40040F17D12023C4F88030C4F88430002028
S31508023E5084F87C0003B030BD6FF07E4300930346BE
S31508023E6000224FF400112046FFF7F1FE0028E4D0A5
S31508023E700320EFE76FF07E4300932B4600224FF4B0
S31508023E8080012046FFF7E3FE0028DBD00320E1E7A6
S31508023E9078B310B50446D0F880300BB32423C4F89F
S31508023EA080302268136823F0010313602046FEF768
S31508023EB0E3FA012813D0A36ABBB92268536823F42C
S31508023EC0904353602268936823F02A03936022681A
S31508023ED0136843F0010313602046FFF7A0FF10BDE5
S31508023EE080F87C30FEF7C4FAD8E72046FFF74AFE88
S31508023EF0E3E701207047000008B5FCF7C1FC094B4F
S31508023F001868094BA3FB00308009FEF78FF90420D5
S31508023F10FEF7A2F9002211464FF0FF30FEF754F9D8
S31508023F2008BD00BF2C040020D34D621008B5FCF76B
S31508023F30E9FD08BD08B5FCF7D9FDFEF79EF908BDEF
S31508023F4008B5002280210248FEF78CFA08BD00BF98
S31508023F500004025810B5FFF7E9FF0E4B1B68C31A97
S31508023F60B3F5FA7F0CD304460B4B1B784BB90122E7
S31508023F70094B1A7080210948FEF774FA054B1C6032
S31508023F8010BD0022044B1A7080210448FEF76AFA13
S31508023F90F4E700BF5C04002058040020000402581D
S31508023FA0014A024B9A6070470000020800ED00E0E1
S31508023FB000B59DB04C22002109A8FCF737FB202248
S31508023FC0002101A8FCF732FB0220FDF741FB002382
S31508023FD00093254B9A6942F440429A619B6903F41D
S31508023FE040430093214BDA6A42F00102DA62DB6A45
S31508023FF003F001030093009B1B4B9B6913F4005FBC
S31508024000FAD0012309934FF4A0230A9302231293A9
S315080240101393042214924FF4F07115911693179282
S315080240201893199200231A931B9309A8FDF73AFBD2
S3150802403000B1FEE73F230193032302930023039370
S31508024040082304934023059306934FF4806207924C
S31508024050089304210DEB0100FDF714FF00B1FEE7FA
S315080240601DB05DF804FB00BF004802580004005862
S3150802407008B5FFF795FFFCF70BFDFFF799FFFFF76A
S315080240803BFFFFF75DFF08BD08B5FFF7F1FF00F03C
S3150802409055F9FFF75FFF00F0DBF9FAE7F0B58DB0E7
S315080240A04D4BD3F8F42042F00202C3F8F420D3F8B9
S315080240B0F42002F002020192019AD3F8E02042F0BB
S315080240C00202C3F8E020D3F8E02002F002020292CC
S315080240D0029AD3F8E02042F00402C3F8E020D3F8AB
S315080240E0E02002F004020392039AD3F8E02042F099
S315080240F00802C3F8E020D3F8E02002F0080204928E
S31508024100049AD3F8E82042F48022C3F8E820D3F8C8
S31508024110E82002F480220592059AD3F8EC2042F4AC
S315080241208072C3F8EC20D3F8EC3003F4807306935C
S31508024130069B0320FEF736F8002211466FF00B00A5
S31508024140FEF742F8002211466FF00A00FEF73CF825
S31508024150002211466FF00900FEF736F800221146D2
S315080241606FF00400FEF730F8002211466FF00300E4
S31508024170FEF72AF8002211466FF00100FEF724F82E
S31508024180002211464FF0FF30FEF71EF880230793F0
S3150802419001230893002409940A94104D07A9284676
S315080241A0FEF770F84FF440770797022608960994A7
S315080241B00A9407230B9307A90948FEF763F807979A
S315080241C0089609940A9409230B9307A92846FEF729
S315080241D059F80DB0F0BD00BF004402580004025859
S315080241E0000C0258F0B4002401E00134E4B2112CA8
S315080241F020D8124D15F8147005EB440595F801C040
S3150802420007EB0C0606FB00064FF4FA55B5FBF6F566
S3150802421006FB05F5B5F5FA5FE7D1B5FBF6F60E80AE
S31508024220013EB6B2B6F5007FDFD2177083F800C03A
S31508024230012000E00020F0BC704700BF00450208DC
S3150802424008B50948094B03604FF4614343600023EC
S315080242508360C36003610C2242618361C3610362A6
S315080242608362FFF715FE08BD0005002000480040DE
S3150802427070B58CB00025ADF82E508DF82D508DF8FE
S315080242802C500BAB0DF12D020DF12E014FF4FA70E5
S31508024290FFF7A8FF204C214B2360A560E5600126A5
S315080242A026746574A574BDF82E306361A6619DF8FF
S315080242B02D30E3619DF82C3023626662A662E662BF
S315080242C026636563A663E563266404236364A564BB
S315080242D0E36425656365A565E56525666566A36682
S315080242E02046FCF717FF039504950596069640F2B5
S315080242F0676307930893099503A92046FDF754F8BF
S3150802430000963346022211462046FDF790F82046CB
S31508024310FDF7A9F80CB070BD6004002000A00040AB
S3150802432008B50023012201460348FFF7E3FC08B15A
S31508024330002008BD0120FCE70005002008B5FFF7AC
S315080243407FFFFFF795FF08BDBFF34F8F0549CA6880
S3150802435002F4E062044B1343CB60BFF34F8F00BFF6
S31508024360FDE700BF00ED00E00400FA0508B5214BA1
S315080243701B78B3B92048FFF7D3FF012800D008BD40
S315080243801D4B1B78013BDBB23F2BF8D8FFF7CEFD5E
S315080243901A4B1860174B01221A70194B00221A7011
S315080243A0EDE7174B1B78013313481844FFF7B8FF9C
S315080243B0012813D1124A13780133DBB213700E4A5D
S315080243C012789342DBD10B4A002111700A4A5278BD
S315080243D0FF2AD4D1022BD2D1FFF7B6FFFFF7A6FDEB
S315080243E0064B1B6864339842C9D9024B00221A70DD
S315080243F0C5E700BFCD0500208C050020D0050020AA
S31508024400CE05002000B58DB040211048FDF712F9FF
S3150802441010B90DB05DF804FB6B4602AA40210B48A1
S31508024420FDF73CF80028F4D1029A40F267639A42F3
S31508024430EFD1039B002BECD19DF816209DF8003096
S31508024440FF2BE6D1022AE4D1FFF77EFF60040020A3
S3150802445008B5FFF78BFFFFF7D5FF08BD0A4491425F
S3150802446000F1FF3300D1704710B511F8014B03F87C
S31508024470014F9142F9D110BDF8B500BFF8BC08BC8E
S315080244809E467047F8B500BFF8BC08BC9E46704702
S31508024490000000000000000000000000000000000C
S315080244A000000000010000000200000003000000F6
S315080244B004000000000000000500000000000000E3
S315080244C000000000000000000600000000000000D6
S315080244D000000000000000000700000000000020A5
S315080244E0000000000102030401020304060708098A
S315080244F00001020304050607080C101418203040B0
S3150802450005020602060307030803090309040A0447
S315080245100B040C040C050D050E050F050F061006F7
S309080245201007100858
S30D08024524ECBDFF7F0100000057
S30D0802452CCD060208C5020208C9
S30908024534A1020208C6
S3150802453800000000EC02002054030020BC030020FF
S315080245480000000000000000000000000000000053
S315080245580000000000000000000000000000000043
S315080245680000000000000000000000000000000033
S315080245780000000000000000000000000000000023
S315080245880000000000000000000000000000000013
S315080245980000000000000000000000000000000003
S315080245A800000000000000000000000000000000F3
S315080245B800000000000000000000000000000000E3
S315080245C800000000000000000000000000000000D3
S315080245D800000000000000000100000000000000C2
S315080245E80E33CDAB34126DE6ECDE05000B00000087
S315080245F800000000000000000000000000000000A3
S315080246080000000000000000000000000000000092
S315080246180000000000000000000000000000000082
S315080246280000000000000000000000000000000072
S315080249580000000000000000D40500200090D003E3
S311080249680090D0030100000010000000BF
S705080207B138
